:100000008A110A120528000009000730990083169A
:10001000051085100511851505168312BC30A0004A
:100020000230A1009C21851916281A281F3083054B
:10003000051E25281030A0002730A1009C2110307B
:10004000A0002730A1009C2113281F3083054520E4
:10005000AC012C081E3C031C4128AD012D083B3C83
:10006000031C3B28E830A0000330A1009C21013094
:10007000AD07031C2E281F3083050130AC07031C7D
:1000800029281F3083050E28442805145830A00065
:100090000230A1009C21D0204421C2204421F8201C
:1000A000442176204421B82044219B2044212B2147
:1000B0004421B42044214421C22044216E20442103
:1000C000B4204421862044216E204421B820903061
:1000D000A0000130A1009C210510080068217921B1
:1000E00008007921682168216821080079216821A8
:1000F0007921682108007921682168210800682198
:100100000800682168217921682108007921792176
:100110006821080068216821682168210800682199
:100120006821080068217921792179210800792145
:100130006821792108006821792168216821080057
:100140007921792108007921682108007921792114
:100150007921080068217921792168210800792115
:100160007921682179210800682179216821080016
:100170006821682168210800792108006821682128
:100180007921080068216821682179210800682107
:1001900079217921080079216821682179210800D5
:1001A0007921682179217921080079217921682133
:1001B00068210800792179217921792179210800A4
:1001C0006821792179217921792108006821682124
:1001D0007921792179210800682168216821792114
:1001E00079210800682168216821682179210800A7
:1001F0006821682168216821682108007921682127
:100200006821682168210800792179216821682105
:100210006821080079217921792168216821080065
:1002200079217921792179216821080068217921B2
:1002300068217921682179210800792179216821B3
:1002400068217921792108006821682179217921A3
:1002500068216821080079216821682179216821B5
:100260000800792168216821682179210800792115
:10027000682168216821682179210800051164300E
:10028000A000A1019C21080005116430A000A1017B
:100290009C216430A000A1019C216430A000A10138
:1002A0009C21080005116430A000A1019C2164304C
:1002B000A000A1019C216430A000A1019C21643018
:1002C000A000A1019C216430A000A1019C21080094
:1002D0000515053084000230AA009930A0000230D4
:1002E000A1004430A2000030A300D72105113E2117
:1002F00008000515053084000230AA009930A000DE
:100300000230A1000E30A2000130A300D721051158
:100310003E2108000515053084000230AA009930FE
:10032000A0000230A100EE30A2000230A300D721CD
:1003300005113E2108009B29A0080319A729AE2119
:10034000A003000000000000000000009C29A1089C
:1003500003190800AE21A103A0039C290C30A500BD
:10036000A50BB029000000001230A200A20BBD298D
:10037000BF21BF21000000000800BF21B6290D30B9
:10038000A400A40BC129000008001030A80200013D
:10039000031C013EA902031C0800CE290A30A80252
:1003A0000001031C013EA902031C0800CE292A08F3
:1003B00080042008A8002108A900C5210130A2025C
:1003C000031CA3032A0980052008A8002108A9000E
:1003D000C521A208031DD729A308031DD72908009A
:02400E00C431BB
:00000001FF
